:100000000C9484000C94A3000C94A3000C94A30003
:100010000C94A3000C94A3000C9499010C94A300DD
:100020000C94A3000C94A3000C94A3000C94A300C4
:100030000C94A3000C94A3000C94A3000C94A300B4
:100040000C94A3000C94A3000C94A3000C94A300A4
:100050000C94190A0C94A3000C94A3000C94A30014
:100060000C94A3000C947A110C94B3060C94A30086
:100070000C94A3000C94A3000C94A3000C94A30074
:100080000C94A3000C94A3000C94A3000C94850A78
:100090000C94D1120C946F060C94A3000C94A30042
:1000A0000C94A3000C94A3000C9420010C94A300C6
:1000B0000C94A3000C94A3000C94A3000C94A30034
:1000C0000C94A3000C94A3000C94A300494E464941
:1000D0004E4954594E414ECDCCCC3D0AD7233C1706
:1000E000B7D13877CC2B329595E6241FB14F0A0053
:1000F0000020410000C84200401C4620BCBE4CCA43
:100100001B0E5AAEC59D740011241FBECFEFD1E265
:10011000DEBFCDBF1DE0A0E0B2E0E2EFFEE400E014
:100120000BBF02C007900D92A433B107D9F710E1BD
:10013000A4E3BDE001C01D92AB3EB107E1F70E9410
:10014000551D0C9477270C9400008A3010F480938E
:10015000390E08951092350E1092360E1092370E09
:100160001092380E08951092350E1092360E10929D
:10017000370E1092380E1092390E10923A0E4FEF41
:100180004093770E30E13093780E21E02093790E82
:1001900088E998E090937B0E80937A0E10927C0E03
:1001A00040937D0E30937E0E20937F0E9093810EB0
:1001B0008093800E3093820E20933B0E10923C0E63
:1001C0001092860E80E090E0FC01EE0FFF1FE35CD2
:1001D000F14F11821082019688309105A9F780E0D5
:1001E00090E0FC01EB5CF14F808F01968830910527
:1001F000C1F780E090E024E6FC01EB5CF14F20A326
:10020000019688309105C1F78FEF9FE390936E0EB2
:1002100080936D0E9093700E80936F0E88E08093A4
:10022000710E8FEF9FE19093730E8093720E8CE2AC
:1002300091E09093750E8093740E1092760E08954F
:100240001F920F920FB60F920BB60F9211242F939D
:100250003F934F935F936F937F938F939F93AF934E
:10026000BF93EF93FF931092A5001092A4002091EA
:10027000220230912302E0913A0E8091AB0DF0E022
:1002800044E0EE0FFF1F4A95E1F7E80FF11DEC5D2A
:10029000FD4F8081280F311D3093A9002093A800C5
:1002A0008091380D863034F08FEF90E09093A90064
:1002B0008093A800A8950E9420110E94FA03E09163
:1002C000390E8091AB0DF0E034E0EE0FFF1F3A9550
:1002D000E1F7E80FF11DEC53FD4F81E060810E94D2
:1002E000110480E293E00197F1F78091380D8F5F60
:1002F0008093380D86E00E948B048F718093390DB6
:100300006091380D4091AB0D0E942211FF91EF9149
:10031000BF91AF919F918F917F916F915F914F911D
:100320003F912F910F900BBE0F900FBE0F901F901B
:1003300018951F920F920FB60F920BB60F921124C1
:10034000EF920F932F933F934F935F936F937F930E
:100350008F939F93AF93BF93EF93FF93DF93CF93CD
:1003600000D0CDB7DEB719821A828FE00E948B04CD
:10037000A89582FF07C086E00E948B048F7180934E
:10038000A80D2AC183FF28C18091A90D9091AA0DC3
:10039000019709F002C18BE39DE06CE6AE014E5F70
:1003A0005F4F9E012F5F3F4F0E940C05882309F489
:1003B00013C18981882309F40FC12091350E309132
:1003C000360E4091370E5091380E80913B0D909132
:1003D0003C0DA0913D0DB0913E0D82179307A407EF
:1003E000B50709F088C08091A4009091A500909372
:1003F000370D8093360D1092A5001092A4008091C5
:10040000380D882331F48CE390E09093230280939D
:1004100022028091220290912302E0913A0E2091D3
:10042000AB0D0A96F0E0B4E0EE0FFF1FBA95E1F7CE
:10043000E20FF11DEC5DFD4F2081820F911D909325
:10044000A9008093A800A8950E941E110091380D64
:10045000E090AB0D8BE39DE06091A80D4091A70D5E
:100460002A810E94E113082F86E00E948B048F717D
:100470008093A70D8430F8F40023E9F0E091390E61
:100480008091AB0DF0E0A4E0EE0FFF1FAA95E1F71D
:10049000E80FF11DEC53FD4F82E060810E941104D2
:1004A00080E293E00197F1F78BE39DE0602F70E02D
:1004B0000E94080419C00E94FA03E091390E80914D
:1004C000AB0DF0E074E0EE0FFF1F7A95E1F7E80F57
:1004D000F11DEC53FD4F81E060810E94110480E228
:1004E00093E00197F1F7A8958091380D80933A0D2C
:1004F0001092380D71C08091350E9091360EA091FA
:10050000370EB091380E0097A105B10509F064C00F
:100510008091A80D853008F45FC0A8950E941E1137
:100520008091350E9091360EA091370EB091380E15
:1005300020913B0D30913C0D40913D0D50913E0D71
:1005400082179307A407B50771F080913F0D815082
:10055000823048F42093350E3093360E4093370E98
:100560005093380EA8950E94FA03E091390E8091BD
:10057000AB0DF0E064E0EE0FFF1F6A95E1F7E80FC6
:10058000F11DEC53FD4F81E060810E94110480E277
:1005900093E00197F1F7A8951FC00E94FA03E0913C
:1005A000390E8091AB0DF0E054E0EE0FFF1F5A952D
:1005B000E1F7E80FF11DEC53FD4F81E060810E94EF
:1005C000110480E293E00197F1F7A89586E00E947C
:1005D0008B048F718093A70D0F900F90CF91DF91B7
:1005E000FF91EF91BF91AF919F918F917F916F910B
:1005F0005F914F913F912F910F91EF900F900BBE14
:100600000F900FBE0F901F901895DF93CF9300D0DF
:1006100000D0CDB7DEB789E492E0A0E0B0E08983F6
:100620009A83AB83BC83CE01019660E070E044E026
:1006300050E00E94692585E39EE064E070E042E5B9
:1006400050E00E9469250F900F900F900F90CF916E
:10065000DF910895EF92FF920F93DF93CF93CDB781
:10066000DEB768970FB6F894DEBF0FBECDBF198214
:100670001A821B821C820E94B300CE01019660E0A8
:1006800070E044E050E00E94592589819A81AB8155
:10069000BC8105E0E02EF12CEC0EFD1E8954924049
:1006A000A040B040D1F485E39EE064E070E042E514
:1006B00050E00E94592580E092E00E946A08209153
:1006C000350E3091360E4091370E5091380EC701DD
:1006D000B90140E020E001E018C080E192E00E9412
:1006E0006A0869817A81C70140E020E001E00E9448
:1006F000F706C7010E946A0880E292E00E946A0839
:10070000C70169E472E040E020E00E94F706C701FB
:100710000E946A088DE092E00E946A0868960FB60F
:10072000F894DEBF0FBECDBFCF91DF910F91FF9048
:10073000EF9008958AEF90E0909323028093220235
:100740000E942A038091390E8A3010F48093390E6A
:100750000E9436040E94FA03E091390E8091AB0D9D
:10076000F0E094E0EE0FFF1F9A95E1F7E80FF11D1E
:10077000EC53FD4F81E060810E94110485E06FE041
:1007800040E020E00E94AF040E94D5031092A50033
:100790001092A40080912202909123029093A900CC
:1007A0008093A8000E941E1108951092A500109237
:1007B000A4001092A00085E08093A1008FEF90E04C
:1007C0009093A9008093A800E2E7F0E08081826026
:1007D00080837894089594B7977F94BFE0E6F0E023
:1007E00090819861908387708860808384B7877FC9
:1007F00084BF08958091AB0D8F3030F48091AB0DA4
:100800008F5F8093AB0D02C01092AB0D80E0089516
:100810009C01862FB9010E9464052C9A2C9880E0D7
:1008200008951F93182F262F88E06FE140E00E9463
:10083000AF04812F90E09093AA0D8093A90D113001
:1008400019F482E066E008C085E060E847E021E056
:100850000E94AF0482E069E00E947C048EE06CE0BC
:100860000E947C04789480E01F9108950F931F9359
:1008700084E00E9457040CEF13E0C8010197F1F7E0
:1008800017982C988CE090E00197F1F7179A82E086
:1008900068E00E947C04C8010197F1F781E06FE1F4
:1008A00040E00E949C0480E01F910F9108950F9AF0
:1008B000249A95B1936095B994B1976094B92398AF
:1008C00090E59CBD9CB59C7F9CBD9DB59E7F9DBDCC
:1008D0002CB5982F9370922B9CBD9DB586958695CF
:1008E0008170982B9DBDEAE6F0E080818C6080836A
:1008F00080E28CBBED9A0895806C9FB7F89428989D
:100900008EBD0DB407FEFDCF6EBD0DB407FEFDCF4D
:10091000289A9FBF08958F7380689FB7F89428988E
:100920008EBD0DB407FEFDCF8EBD0DB407FEFDCF0D
:100930008EB5289A9FBF0895FF920F931F93062F9D
:10094000F42E0E948B04082310E002C01595079531
:10095000FA94E2F7802F1F910F91FF900895DF9294
:10096000EF92FF920F931F93D82EF62EE42E022FB4
:100970000E948B046F2D6095682310E002C0000F69
:10098000111FEA94E2F7F0226F298D2D0E947C045A
:100990001F910F91FF90EF90DF900895CB01089584
:1009A000FC01DA015FB7F894289880E28EBD0DB49F
:1009B00007FEFDCF1EBC0DB407FEFDCF4EB564177C
:1009C00030F1942F20E030E01EBC0DB407FEFDCFC7
:1009D0008EB52827022E2295207F2025032E322F28
:1009E00022952F700226269532272327220F220FC9
:1009F000220F20258083915011F03196E5CF10977A
:100A000039F01C92232B21F481E08C9301C04068C3
:100A1000289A5FBF842F0895FF920F931F93CF935F
:100A2000DF938C01EA01D901FFB6F894289880E29F
:100A30008EBD0DB407FEFDCF1EBC0DB407FEFDCF6D
:100A40009EB5691708F436C020E030E040E050E081
:100A5000692F70E01CC01EBC0DB407FEFDCF8EB523
:100A6000F801E20FF31F80834827042E4295407F50
:100A70004025052E542F42954F7004264695542745
:100A80004527440F440F440F40252F5F3F4F261743
:100A9000370708F3109729F01C92452B11F481E0D9
:100AA0008C93209741F01EBC0DB407FEFDCF8EB590
:100AB000888301C09068289AFFBE892FDF91CF916B
:100AC0001F910F91FF900895982FFB012FB7F89475
:100AD000289880E68EBD0DB407FEFDCF9EBD0DB4F7
:100AE00007FEFDCF80818EBD915011F03196F7CF7A
:100AF0000DB407FEFDCF289A2FBF0895FC01DA013F
:100B00003FB7F894289880E28EBD0DB407FEFDCF64
:100B10001EBC0DB407FEFDCF2EB56217A0F0922FBC
:100B20001EBC0DB407FEFDCF8EB58083915011F031
:100B30003196F6CF109741F01EBC0DB407FEFDCFE5
:100B40008EB58C9301C02068289A3FBF822F0895EC
:100B5000833309F080E0089583E30895E82FF0E0FF
:100B6000EE0FFF1FE357F14F20813181C901089536
:100B7000E82FF0E0EE0FFF1FE357F14F11821082D4
:100B800008959B01AC01529A53985A9A5B9A64E07B
:100B9000220F331F441F551F6A95D1F760E072E1A1
:100BA0008AE790E00E94A924215030401092CD00A5
:100BB0002093CC0080E48093C80088E98093C9002A
:100BC00086E08093CA00789408959B01AC01689AEE
:100BD0006998709A719A74E0220F331F441F551F51
:100BE0007A95D1F760E072E18AE790E00E94A9244B
:100BF000215030401092C5002093C40080E48093BF
:100C0000C00088E98093C10086E08093C200789498
:100C10000895FC0180918A0E8823D1F4F0938C0E04
:100C2000E0938B0E60938A0E20918F0E3091900E80
:100C3000808190E0822793279093900E80938F0E6F
:100C400080818093CE008091C90080628093C9002A
:100C500080918A0E8823E1F70895FC018091870E28
:100C60008823D1F4F093890EE093880E6093870E69
:100C700020918D0E30918E0E808190E082279327F7
:100C800090938E0E80938D0E80818093C60080910C
:100C9000C10080628093C1008091870E8823E1F7B4
:100CA0000895DF93CF930F92CDB7DEB78983CE013E
:100CB000019661E00E942D060F90CF91DF9108957B
:100CC000DF93CF930F92CDB7DEB78983CE01019624
:100CD00061E00E9409060F90CF91DF9108951F9265
:100CE0000F920FB60F920BB60F9211242F933F93D2
:100CF0008F939F93EF93FF93E0918B0EF0918C0E67
:100D00003196F0938C0EE0938B0E319780918A0E82
:100D1000815080938A0E80918A0E882391F0809171
:100D20008F0E9091900E2181332727FD3095282733
:100D300039273093900E20938F0E81818093CE00BF
:100D400005C08091C9008F7D8093C900FF91EF910C
:100D50009F918F913F912F910F900BBE0F900FBEDF
:100D60000F901F9018951F920F920FB60F920BB60F
:100D70000F9211242F933F938F939F93EF93FF93A1
:100D8000E091880EF091890E3196F093890EE093F0
:100D9000880E31978091870E81508093870E8091C5
:100DA000870E882391F080918D0E90918E0E218177
:100DB000332727FD30952827392730938E0E20932F
:100DC0008D0E81818093C60005C08091C1008F7D0A
:100DD0008093C100FF91EF919F918F913F912F914F
:100DE0000F900BBE0F900FBE0F901F901895BF92E3
:100DF000CF92DF92EF92FF920F931F93DF93CF93E7
:100E0000CDB7DEB72C970FB6F894DEBF0FBECDBFBF
:100E10006C01FB01B42EE22E77FD02C0FF2408C056
:100E2000F095E195FF4F8DE2D6018C93FF24F3946A
:100E300040E08E010F5F1F4F10C0200F311FCF0108
:100E40006AE070E00E949624805DD9018C93CF0106
:100E50006AE070E00E949624FB01242F30E04F5F8F
:100E6000EA30F10554F7020F131F8E2F805DF80151
:100E70008083642FCE01019620E305C0FC01E60FBC
:100E8000F11D20836F5FE616C8F76B15B8F3862F48
:100E900090E09E012F5F3F4FF901E80FF91F10828C
:100EA0000197D901A80FB91F019640E050E08C01CD
:100EB0002E2D30E07EE214C0C801841B950B8217F2
:100EC000930729F4F601EF0DF11D7083F394F601F9
:100ED000EF0DF11D8C918083F3944F5F5F4F11975D
:100EE000461750F3F601EF0DF11D1082C6012C9646
:100EF0000FB6F894DEBF0FBECDBFCF91DF911F912B
:100F00000F91FF90EF90DF90CF90BF9008954F9298
:100F10005F926F927F928F929F92AF92BF92CF9289
:100F2000DF92EF92FF920F931F93DF93CF93CDB792
:100F3000DEB72C970FB6F894DEBF0FBECDBF3C01D5
:100F40006A017B01422E502E77FD02C099240DC00C
:100F5000F094E094D094C094C11CD11CE11CF11C0D
:100F60008DE2F30180839924939488245E01089490
:100F7000A11CB11C19C00A0D1B1DC701B6012AE036
:100F800030E040E050E00E94CB24605DF8016083D7
:100F9000C701B6012AE030E040E050E00E94CB24D7
:100FA000C901DA016C017D01082D10E08394FAE09B
:100FB000CF16D104E104F104F4F6A00EB11E8C2D7D
:100FC000805DF5018083482DCE01019620E305C0A8
:100FD000FC01E40FF11D20834F5F5416C8F7441540
:100FE000B8F3842F90E09E012F5F3F4FF901E80F87
:100FF000F91F10820197D901A80FB91F019620E0AF
:1010000030E0BC01052D10E05EE214C0CB01821B74
:10101000930B8017910729F4F301E90DF11D50831B
:101020009394F301E90DF11D8C91808393942F5FCC
:101030003F4F1197241750F3F301E90DF11D108272
:10104000C3012C960FB6F894DEBF0FBECDBFCF9173
:10105000DF911F910F91FF90EF90DF90CF90BF90A5
:10106000AF909F908F907F906F905F904F9008957A
:10107000DC010D900020E9F71197A81BB90B6A2F2E
:101080000E942D060895EF92FF920F93DF93CF9366
:10109000CDB7DEB72A970FB6F894DEBF0FBECDBF2F
:1010A000BC017E010894E11CF11CC70140E020E076
:1010B00001E00E94F706C7010E9438082A960FB681
:1010C000F894DEBF0FBECDBFCF91DF910F91FF909F
:1010D000EF900895DC010D900020E9F71197A81B0F
:1010E000B90B6A2F0E9409060895CF92DF92EF9202
:1010F0000F93DF93CF93CDB7DEB72A970FB6F8944F
:10110000DEBF0FBECDBFAB01BC016E010894C11C98
:10111000D11CC60120E000E0EE24E3940E94870782
:10112000C6010E946A082A960FB6F894DEBF0FBE69
:10113000CDBFCF91DF910F91EF90DF90CF900895C9
:10114000EF92FF920F93DF93CF93CDB7DEB72A973D
:101150000FB6F894DEBF0FBECDBFBC017E01089470
:10116000E11CF11CC70140E020E001E00E94F7060D
:10117000C7010E946A082A960FB6F894DEBF0FBE18
:10118000CDBFCF91DF910F91FF90EF9008958098A0
:1011900081988298839886E880937A0080E480938F
:1011A0007C000895806480937C0086E880937A00B8
:1011B00080917A00806480937A0080917A0084FF25
:1011C000FCCF2091780030917900C9010895609199
:1011D0007A0E70917B0E660F771F660F771F409116
:1011E000AD0D8091780E481798F480917C0EE42F15
:1011F000F0E0E80FF11DEE0FFF1FEF56F14F808179
:10120000918162E070E00E9496246059784E0CC093
:101210008091790E823061F48091780E90E0242FD5
:1012200030E08217930724F04F5F4093AD0D02C06A
:101230001092AD0DCB0108956091800E7091810EDA
:10124000660F771F660F771F4091AC0D80917E0E61
:10125000481798F48091820EE42FF0E0E80FF11D1A
:10126000EE0FFF1FEF56F14F8081918162E070E039
:101270000E9496246059784E0CC080917F0E823077
:1012800061F480917E0E90E0242F30E08217930766
:1012900024F04F5F4093AC0D02C01092AC0DCB0117
:1012A000089510928500109284001092950010927B
:1012B000940008959091770EE82FF0E0EC59FC4FE0
:1012C000E0819E1709F44FC080917D0E8E1709F4BE
:1012D0004AC0E23029F1E33030F4EE2349F0E13046
:1012E00009F041C011C0E33039F1E430E1F530C01C
:1012F000CB0162E070E00E9496246059784E7093B2
:101300008900609388000895CB0162E070E00E943C
:1013100096246059784E70938B0060938A000895EC
:10132000CB0162E070E00E9496246059784E709381
:101330008D0060938C000895CB0162E070E00E9404
:1013400096246059784E70939900609398000895A0
:10135000CB0162E070E00E9496246059784E709351
:101360009B0060939A000895CF93DF93259A269A65
:10137000279AE0E8F0E01082A1E8B0E01C9226E8AD
:1013800030E0E901198218828081826080838C912B
:1013900080618C938081886A80838C9181608C933A
:1013A00060E070EF7983688320E737E1309389004C
:1013B0002093880030938B0020938A0030938D0017
:1013C00020938C00EFE6F0E08081816080836C9A4E
:1013D0006B9AE0E9F0E01082A1E9B0E01C9246E9E6
:1013E00050E0EA01198218828081826080838C91AA
:1013F00080618C938081886A80838C9181608C93DA
:1014000079836883309399002093980030939B00F0
:1014100020939A0088EE9DEF90939500809394001E
:10142000E1E7F0E08081816080837894DF91CF9163
:1014300008951F920F920FB60F920BB60F921124C0
:101440002F933F934F935F936F937F938F939F93CC
:10145000AF93BF93EF93FF9380916D0E90916E0EBB
:10146000880F991F880F991F90938700809386009B
:101470008091770E813061F0813018F08230A9F4CC
:101480000EC00E94E70890938900809388000DC0E9
:101490000E94E70890938B0080938A0006C00E9408
:1014A000E70890938D0080938C0080917D0E8130B1
:1014B00061F0813018F08230A9F40EC00E941C093E
:1014C00090938900809388000DC00E941C0990931E
:1014D0008B0080938A0006C00E941C0990938D00A7
:1014E00080938C00FF91EF91BF91AF919F918F916D
:1014F0007F916F915F914F913F912F910F900BBE14
:101500000F900FBE0F901F9018951F920F920FB65D
:101510000F920BB60F9211242F933F934F935F932B
:101520006F937F938F939F93AF93BF93EF93FF93AB
:1015300080916F0E9091700E880F991F880F991FE0
:1015400090939700809396008091770E833019F0E6
:10155000843071F407C00E94E7089093990080934B
:10156000980006C00E94E70890939B0080939A0021
:1015700080917D0E833019F0843071F407C00E9491
:101580001C09909399008093980006C00E941C0942
:1015900090939B0080939A00FF91EF91BF91AF9140
:1015A0009F918F917F916F915F914F913F912F917B
:1015B0000F900BBE0F900FBE0F901F901895519A71
:1015C000509A599A589AE9EBF0E0808183608083C1
:1015D00080E28093B80084E08093BC00089584EAA0
:1015E0008093BC00089584E98093BC00089520E0B6
:1015F00030E002C02F5F3F4F8091BC0087FD06C0E6
:1016000083E228323807B1F780E0089580E028525D
:10161000334208F481E008958093BB0084E880930E
:10162000BC000895813029F48091BC008F70806CDB
:1016300004C08091BC008F7080688093BC000895C6
:101640008091BB0008958091B9000895EF92FF92B8
:101650000F931F93CF93DF93182FE62E042FF52EB1
:1016600084EA8093BC000E94F70A1093BB0084E8D0
:101670008093BC000E94F70A8091B9008871B1F490
:10168000802F9F2D9C01E90110E004E808C089919A
:101690008093BB000093BC000E94F70A1F5F1E15D9
:1016A000B0F384E98093BC0081E004C084E98093B6
:1016B000BC0080E0DF91CF911F910F91FF90EF90E0
:1016C00008950F931F93182F062F84EA8093BC0070
:1016D0000E94F70A1093BB0014E81093BC000E940C
:1016E000F70A8091B900887159F00093BB001093FC
:1016F000BC000E94F70A84E98093BC0081E004C02A
:1017000084E98093BC0080E01F910F910895FF92BF
:101710000F931F93182F062FF42E84EA8093BC009A
:101720000E94F70A1093BB0014E81093BC000E94BB
:10173000F70A8091B900887189F00093BB0010937B
:10174000BC000E94F70AF092BB001093BC000E94FC
:10175000F70A84E98093BC0081E004C084E98093A7
:10176000BC0080E01F910F91FF900895CF92DF920F
:10177000EF92FF921F93CF93DF93182FF62E6A01FB
:1017800084EA8093BC000E94F70A1F5F1093BB009D
:1017900084E88093BC000E94F70A8091B9008871A8
:1017A00059F510E0CF2DD0E021970CC081E00E94C8
:1017B000120B0E94F70A8091BB00F70180830E9400
:1017C000F70A1F5F812F90E07601E80EF91E8C1753
:1017D0009D0764F380E00E94120B0E94F70A80913B
:1017E000BB00F70180830E94F70A84E98093BC0064
:1017F0000E94F70A81E006C084E98093BC000E9441
:10180000F70A80E0DF91CF911F91FF90EF90DF907A
:10181000CF9008950F931F93DF93CF9300D0CDB750
:10182000DEB781E489831A8282E461E08E010F5F72
:101830001F4FA8010E94260B813011F080E006C0E6
:1018400082E462E0A8010E94B60B81E00F900F9045
:10185000CF91DF911F910F9108950F931F93DF9305
:10186000CF9300D0CDB7DEB781E489831A8282E4BA
:1018700061E08E010F5F1F4FA8010E94260B81308F
:1018800029F482E462E0A8010E94B60B998180E00D
:101890002A8130E0282B392BC9010F900F90CF916E
:1018A000DF911F910F9108952F923F924F925F9277
:1018B0006F927F928F929F92AF92BF92CF92DF9260
:1018C000EF92FF920F931F93DF93CF93CDB7DEB7C5
:1018D0002E970FB6F894DEBF0FBECDBFFE01319636
:1018E0008AE0DF011D928A95E9F78EEE64EF4EE201
:1018F0000E94870B813009F588E092E028EC30E007
:10190000F9013197F1F70197D9F78EEE66EF0E9452
:10191000610B813079F48EEE62E0AE014F5F5F4F74
:101920000E94B60B998180E02A81022F10E0082BDB
:10193000192B09C08CE693E002C083E793E00E9474
:101940006A0800E010E08EEE64EF44EF0E94870B1F
:101950008130D1F588E29AE028EC30E0F901319746
:10196000F1F70197D9F78EEE66EF0E94610B813097
:1019700041F58EEE63E0AE014F5F5F4F0E94B60B04
:10198000898190E0A0E0B0E02C01332422248B81F7
:1019900090E0A0E0B0E0282A392A4A2A5B2A9A81FE
:1019A00080E0AA2797FDA095BA2F282A392A4A2A2B
:1019B0005B2A45E055944794379427944A95D1F78C
:1019C0000AC08AE793E002C081E893E00E946A08B7
:1019D000222433242101B801882777FD8095982F90
:1019E0002091BE0D3091BF0D40E050E0621B730BA3
:1019F000840B950B2091BC0D3091BD0D40E050E063
:101A00000E9463247B018C013FE015950795F794B4
:101A1000E7943A95D1F76091C60D7091C70D88276C
:101A200077FD8095982F2BE0660F771F881F991FF1
:101A30002A95D1F72091C80D3091C90D442737FD63
:101A40004095542F2E0D3F1D401F511F0E94CB2447
:101A500059016A01AE0CBF1CC01ED11E88E090E087
:101A6000A0E0B0E0A80EB91ECA1EDB1ED601C5015B
:101A700014E0B595A795979587951A95D1F790930A
:101A8000AF0D8093AE0D88E590EFAFEFBFEFA80EDE
:101A9000B91ECA1EDB1EC601B501A60195010E9432
:101AA00063243B014C01ACE0959487947794679450
:101AB000AA95D1F72091B80D3091B90D442737FD83
:101AC0004095542FC601B5010E9463247B018C010F
:101AD000FDE015950795F794E794FA95D1F782E024
:101AE00090E0A0E0B0E0E80EF91E0A1F1B1F209155
:101AF000C00D3091C10D442737FD4095542FC401CE
:101B0000B3010E946324BC01992777FD9095892F2A
:101B1000E60EF71E081F191F52E015950795F7945A
:101B2000E7945A95D1F780E090E8A0E0B0E0E80EA5
:101B3000F91E0A1F1B1F2091BA0D3091BB0D40E00A
:101B400050E0C801B7010E946324DC01CB014FE0E3
:101B5000B695A795979587954A95D1F78B879C87DA
:101B6000AD87BE872091B60D3091B70D442737FD64
:101B70004095542FC601B5010E9463247B018C015E
:101B80003BE015950795F794E7943A95D1F7809146
:101B9000B40D9091B50DAA2797FDA095BA2F22E01C
:101BA000880F991FAA1FBB1F2A95D1F7E80EF91EAF
:101BB0000A1F1B1F2091C20D3091C30D442737FD12
:101BC0004095542FC401B3010E946324ABE0959566
:101BD000879577956795AA95D1F7E60EF71E081FAA
:101BE000191FEE0CFF1C001F111F2E183F08400A82
:101BF000510AC201B1012AE638E140E050E00E94FA
:101C0000632497FD0FC0660F771F881F991F2B85D0
:101C10003C854D855E850E94A924C901DA015C01DD
:101C20006D010CC02B853C854D855E850E94A924E5
:101C300059016A01AA0CBB1CCC1CDD1C5527D7FC22
:101C40005A954D2D3C2D2B2DCA01B9010E946324BC
:101C50002EED3BE040E050E00E9463247B018C01CC
:101C6000C601B50123E433EE4FEF5FEF0E9463241A
:101C7000BC01992777FD9095892F6153714F8F4F44
:101C80009F4F78011127F7FC1095012F6E0D7F1DD6
:101C9000801F911F24E095958795779567952A95E4
:101CA000D1F76A0D7B1D8C1D9D1D6093B00D709347
:101CB000B10D8093B20D9093B30D81E02E960FB6C7
:101CC000F894DEBF0FBECDBFCF91DF911F910F9172
:101CD000FF90EF90DF90CF90BF90AF909F908F904C
:101CE0007F906F905F904F903F902F90089588E87D
:101CF00093E00E946A088091AE0D9091AF0D6AE06A
:101D000070E00E949624882777FD8095982F0E9486
:101D100075088FE893E00E946A088091AE0D90915B
:101D2000AF0D6AE070E00E949624AA2797FDA09567
:101D3000BA2FBC01CD010E94750881E993E00E9491
:101D40006A088091AE0D9091AF0D089584E993E0FB
:101D50000E946A086091B00D7091B10D8091B20D32
:101D60009091B30D0E94750881E993E00E946A0882
:101D70006091B00D7091B10D8091B20D9091B30D45
:101D800008950F931F93DF93CF93CDB7DEB72A97B4
:101D90000FB6F894DEBF0FBECDBF8E010F5F1F4F91
:101DA0008AE0F80111928A95E9F78EEE64EF4EE22F
:101DB0000E94870B813011F080E0DAC18EEE6AEA72
:101DC0000E94610B8EEE62E0A8010E94B60B81308A
:101DD00081F4898190E0A0E0B0E0BA2FA92F982F7C
:101DE00088272A8130E0282B392B3093B50D20939A
:101DF000B40D8EEE6CEA0E94610B8EEE62E0AE01D5
:101E00004F5F5F4F0E94B60B813081F4898190E073
:101E1000A0E0B0E0BA2FA92F982F88272A8130E0C0
:101E2000282B392B3093B70D2093B60D8EEE6EEA2A
:101E30000E94610B8EEE62E0AE014F5F5F4F0E9429
:101E4000B60B813081F4898190E0A0E0B0E0BA2F38
:101E5000A92F982F88272A8130E0282B392B3093FF
:101E6000B90D2093B80D8EEE60EB0E94610B8EEEE3
:101E700062E0AE014F5F5F4F0E94B60B813081F48C
:101E8000898190E0A0E0B0E0BA2FA92F982F882791
:101E90002A8130E0282B392B3093BB0D2093BA0DCB
:101EA0008EEE62EB0E94610B8EEE62E0AE014F5F40
:101EB0005F4F0E94B60B813081F4898190E0A0E0F1
:101EC000B0E0BA2FA92F982F88272A8130E0282B3D
:101ED000392B3093BD0D2093BC0D8EEE64EB0E9428
:101EE000610B8EEE62E0AE014F5F5F4F0E94B60B5A
:101EF000813081F4898190E0A0E0B0E0BA2FA92F71
:101F0000982F88272A8130E0282B392B3093BF0D5A
:101F10002093BE0D8EEE66EB0E94610B8EEE62E0AA
:101F2000AE014F5F5F4F0E94B60B813081F4898113
:101F300090E0A0E0B0E0BA2FA92F982F88272A813F
:101F400030E0282B392B3093C10D2093C00D8EEE3D
:101F500068EB0E94610B8EEE62E0AE014F5F5F4F57
:101F60000E94B60B813081F4898190E0A0E0B0E05E
:101F7000BA2FA92F982F88272A8130E0282B392BB8
:101F80003093C30D2093C20D8EEE6AEB0E94610B5D
:101F90008EEE62E0AE014F5F5F4F0E94B60B813064
:101FA00081F4898190E0A0E0B0E0BA2FA92F982FAA
:101FB00088272A8130E0282B392B3093C50D2093B8
:101FC000C40D8EEE6CEB0E94610B8EEE62E0AE01F2
:101FD0004F5F5F4F0E94B60B813081F4898190E0A2
:101FE000A0E0B0E0BA2FA92F982F88272A8130E0EF
:101FF000282B392B3093C70D2093C60D8EEE6EEB38
:102000000E94610B8EEE62E0AE014F5F5F4F0E9457
:10201000B60B813081F4898190E0A0E0B0E0BA2F66
:10202000A92F982F88272A8130E0282B392B30932D
:10203000C90D2093C80D8BE993E00E946A08609156
:10204000B40D7091B50D882777FD8095982F0E946B
:10205000750882EA93E00E946A086091B60D70915B
:10206000B70D882777FD8095982F0E94750882EA22
:1020700093E00E946A086091B80D7091B90D8827AD
:1020800077FD8095982F0E94750882EA93E00E9460
:102090006A086091BA0D7091BB0D80E090E00E94DB
:1020A000750882EA93E00E946A086091BC0D709105
:1020B000BD0D80E090E00E94750882EA93E00E94E6
:1020C0006A086091BE0D7091BF0D80E090E00E94A3
:1020D000750882EA93E00E946A086091C00D7091D1
:1020E000C10D882777FD8095982F0E94750882EA98
:1020F00093E00E946A086091C20D7091C30D882719
:1021000077FD8095982F0E94750882EA93E00E94DF
:102110006A086091C40D7091C50D882777FD809580
:10212000982F0E94750882EA93E00E946A086091E5
:10213000C60D7091C70D882777FD8095982F0E9456
:10214000750882EA93E00E946A086091C80D709158
:10215000C90D882777FD8095982F0E94750882EA1F
:1021600093E00E946A0881E993E00E946A0881E096
:102170002A960FB6F894DEBF0FBECDBFCF91DF9188
:102180001F910F910895FC018081860F808308952F
:10219000FC018081819580830895FC018081860FF8
:1021A00080830895FC018081819580830895FC01DE
:1021B00080819181860F971F918380830895FC0110
:1021C00080819181909581959F4F9183808308951F
:1021D000FC0180819181860F971F918380830895F0
:1021E000FC0180819181909581959F4F918380839F
:1021F0000895FC01882777FD8095982F20813181F3
:1022000042815381260F371F481F591F2083318376
:10221000428353830895FC0180819181A281B3811F
:10222000B095A095909581959F4FAF4FBF4F8083FC
:102230009183A283B38308959A9A0895A29A0895E8
:10224000A2980895E42FF0E0DF01AF58BF4E1C9232
:10225000DF01A35ABF4E8C93E75BFF4E1082609361
:10226000E40D8091DA0D8A3F28F48091DA0D8F5FBA
:102270008093DA0D6623C1F08091DE0D9091DF0D21
:1022800066956695262F30E0820F931F9093DF0DA1
:102290008093DE0D8091E00D9091E10D280F391FA4
:1022A0003093E10D2093E00D8091DE0D9091DF0DD4
:1022B000855F9140F0F02091E00D3091E10D60914B
:1022C000DE0D7091DF0D84E690E0AC01249FC0012B
:1022D000259F900D349F900D11240E9482246093BD
:1022E000DD0D1092DF0D1092DE0D1092E10D1092B7
:1022F000E00D08951F920F920FB60F920BB60F923A
:102300001124EF92FF920F931F932F933F934F93BC
:102310005F936F937F938F939F93AF93BF93EF934D
:10232000FF939091C6009093E20D8091100E8093E0
:10233000110E80910F0E8093100E80910E0E8093DF
:102340000F0E80910D0E80930E0E90930D0E8091C6
:102350000C0E882349F4943209F00CC181E080937B
:102360000C0E10920B0E06C1813009F041C0209175
:102370000B0E253031F58091F70D823551F48091A7
:10238000F80D8D3401F58091F90D8334E1F482E08C
:102390000BC08734C1F48091F80D873451F48091DB
:1023A000F90D813481F483E080930C0E10920B0EB2
:1023B0001AC0833541F48091F90D813421F484E011
:1023C000F3CF243170F4E22FF0E0EB50F24F908322
:1023D000E22FEF5FE0930B0EF0E0EB50F24F108234
:1023E00002C010920C0E10920A0E1092090EC2C07A
:1023F0008230E1F59D3009F4BBC09C3209F0A9C0E0
:10240000F090090E83E18F1508F4A3C0E0900A0E46
:10241000E4E0EE1639F0F6E0EF1621F082E0E8167F
:1024200009F091C00F2D10E085EF9DE00E9421255D
:10243000000F111F03551F4EF80191838083F39401
:10244000F092090EE5EFFDE090E080818E3249F4D4
:102450000F2D10E0892F90E08A50924F0E94212585
:1024600067C09F5F3196943181F76DC0833009F06A
:1024700047C09D3009F47CC09C3209F06AC0F090DE
:10248000090EF3E1FF1508F464C0E0900A0E85E040
:10249000E81608F458C0E6E0EE1520F4F8E0EF1670
:1024A00009F051C00F2D10E00A5F1F4F85EF9DE02E
:1024B0000E9421259C01000F111F03551F4EF8019A
:1024C00031832083F394F092090E20E030E0822FD4
:1024D000F901EB50F24FE081EE23A9F1EE3251F415
:1024E0000F2D10E00A5F1F4F90E08A50924F0E941C
:1024F00021251EC02F5F3F4F2431310541F723C0F6
:102500008430B1F59D30A1F19C3219F5F090090E9F
:10251000F3E1FF15F0F0E0900A0E81E0E81699F47F
:102520000F2D10E0065F1F4F85EF9DE00E942125D3
:102530009C01000F111F03551F4EF80131832083AA
:10254000F394F092090E10920B0EE394E0920A0EAF
:1025500011C0A0910B0EEA2FF0E0EB50F24F9083E8
:10256000AF5FA0930B0EB0E0AB50B24F1C9202C015
:1025700010920C0EFF91EF91BF91AF919F918F91AF
:102580007F916F915F914F913F912F911F910F918B
:10259000FF90EF900F900BBE0F900FBE0F901F900B
:1025A00018951F920F920FB60F920BB60F9211242F
:1025B0002F933F934F935F936F937F938F939F934B
:1025C000AF93BF93EF93FF93DF93CF9300D000D0EF
:1025D00000D0CDB7DEB75091CE005093E30D90916F
:1025E000F30D9093F40D2091F20D2093F30D3091A3
:1025F000F10D3093F20D4091F00D4093F10D509399
:10260000F00D8091ED0D823001F58091EF0D813359
:1026100009F08DC099832A833B834C835D831E829E
:10262000CE0101960E941D2520E030E040E251E4F9
:102630000E943F210E94691F6115710509F475C050
:102640007093B0106093AF1070C08091ED0D813029
:1026500009F073C08091EF0D823191F499832A8340
:102660003B834C831D821E82CE0101960E94212550
:10267000009709F45CC09093AE108093AD1057C0E2
:10268000873191F499832A833B834C831D821E8278
:10269000CE0101960E942125009709F448C090932D
:1026A000B0108093AF1043C08F3189F499832A838F
:1026B0003B834C835D831E82CE0101960E942125BF
:1026C0000097A9F19093B2108093B11030C084327A
:1026D00089F499832A833B834C835D831E82CE01D8
:1026E00001960E942125009711F19093B4108093D8
:1026F000B3101DC08B32D9F499832A833B834C835A
:102700005D831E82CE0101960E941D2520E030E0EF
:1027100048EC52E40E943F210E94691F6115710537
:1027200021F07093B6106093B5101092ED0D80916A
:10273000EF0D8F5F8093EF0D2CC09734B9F42035E7
:10274000A9F4323541F44D3489F4533479F41092BC
:10275000EF0D81E009C0373449F4473439F451347E
:1027600029F41092EF0D82E08093ED0D8091F30D2E
:10277000823B79F48091F20D853A59F48091F10D04
:10278000853639F45B3429F4F89480E00E94EB0339
:10279000FFCF2696DEBFCDBFCF91DF91FF91EF91A6
:1027A000BF91AF919F918F917F916F915F914F9169
:1027B0003F912F910F900BBE0F900FBE0F901F9067
:1027C0001895CF92DF92EF920F93CF93DF936C0126
:1027D000EE2DF0E0DF01AF58BF4E6C93DF01A35A3E
:1027E000BF4E4C93E75BFF4E20830093E40DFC014A
:1027F00080819181A281B3818093E60D9093E70D52
:10280000A093E80DB093E90D1092DA0D8091DE0DE2
:102810009091DF0D01969093DF0D8093DE0D0023E4
:10282000C1F08091DE0D9091DF0D202F2695269529
:1028300030E0820F931F9093DF0D8093DE0D809127
:10284000E00D9091E10D280F391F3093E10D209399
:10285000E00D8091DE0D9091DF0D855F9140F0F0ED
:102860002091E00D3091E10D6091DE0D7091DF0D52
:1028700084E690E0AC01249FC001259F900D349F19
:10288000900D11240E9482246093DD0D1092DF0DC3
:102890001092DE0D1092E10D1092E00DD60114960B
:1028A0008C911497813009F086C088E08093DC0D0C
:1028B00058968D919C9159979093140E8093130E76
:1028C000E0E010C0F0E0DF011496AA0FBB1FAC0DD2
:1028D000BD1D8D919C91EE0FFF1FEB57FF4E918315
:1028E0008083E22F8091DC0D2E2F2F5FE81750F3AD
:1028F000E093120EF60186818F3F39F48781882399
:1029000021F08093290D1092DB0D1092120E24C03D
:10291000C22FD0E0FE01EE0FFF1FDF01AB57BF4E0D
:102920008D919C91EF56F14F91838083253078F4FF
:10293000CB5CD14FE88DF0E0EE0FFF1FEB57FF4E61
:1029400060817181660F771F822F0E945A098091E2
:10295000120E8F5F8093120E2091120E8091DC0D6B
:102960002817B0F2D60116968C9116978093D00D49
:1029700016968C911697E82FF0E08091DC0D9F0160
:10298000280F311D2034310594F48091DC0DE80FBF
:10299000F11D17968C9124E1829FC00111248C5E59
:1029A0009940EE0FFF1FEF56F14F9183808381E036
:1029B0008093EE0D86C0823009F083C080E1809361
:1029C000DC0DD60198968D919C9199979093140E59
:1029D0008093130EE0E010C0F0E0DF011496AA0F20
:1029E000BB1FAC0DBD1D8D919C91EE0FFF1FEB57D2
:1029F000FF4E91838083E22F8091DC0D2E2F2F5F7D
:102A0000E81750F3E093120EF60186818F3F39F4F8
:102A10008781882321F08093290D1092DB0D10927D
:102A2000120E24C0C22FD0E0FE01EE0FFF1FDF0107
:102A3000AB57BF4E8D919C91EF56F14F91838083A0
:102A4000253078F4CB5CD14FE88DF0E0EE0FFF1F1E
:102A5000EB57FF4E60817181660F771F822F0E94B6
:102A60005A098091120E8F5F8093120E2091120EE0
:102A70008091DC0D2817B0F2D60116968C9116972E
:102A80008093D00D16968C911697E82FF0E08091E8
:102A9000DC0D9F01280F311D2034310594F4809105
:102AA000DC0DE80FF11D17968C9124E1829FC00187
:102AB00011248C5E9940EE0FFF1FEF56F14F91836A
:102AC00080838091130E8093E50D8091CE0D8B3025
:102AD00030F584E0D60114968C9314978091CE0D36
:102AE00015968C93159716961C928091CE0D90E0BA
:102AF0002AE130E0829FF001839FF00D929FF00D5C
:102B00001124EF5EF04F178A6091CE0D8AE1689F25
:102B1000B00111246F5E704FC601089614C08091F9
:102B2000CE0D8C3028F584E0D60114968C93149742
:102B30008091CE0D15968C93159716961C92C60112
:102B4000089669EA73E00E944A258091130E9091DD
:102B5000140EF60191A380A301969093140E809316
:102B6000130E8091CE0D8F5F8093CE0D84E2D4C082
:102B70008091CE0D8F5F8093CE0D8150853110F006
:102B80001092CE0D83E0D60114968C931497809109
:102B90002A0D15968C9315978091130E9091140E13
:102BA00019969C938E93189701969093140E809388
:102BB000130E80912A0D813188F4893008F070C09D
:102BC0008330A9F1843030F48130F1F0823009F0A3
:102BD00098C01EC0843009F05EC042C0833109F441
:102BE00077C0843138F4813109F465C0823109F04D
:102BF00088C069C0853109F475C0853108F46DC09D
:102C0000863109F07EC073C0F601068317827EC04C
:102C100020E030E090E008C0E92FF0E0EF58FF4EF0
:102C20008081280F311D9F5F9031B0F327C020E0D5
:102C300030E090E008C0E92FF0E0E35AFF4E8081D9
:102C4000280F311D9F5F9031B0F39093120E74E006
:102C5000369527957A95E1F7F6013783268356C096
:102C600020E030E090E008C0E92FF0E0E75BFF4EA5
:102C70008081280F311D9F5F9031B0F39093120E29
:102C800064E0369527956A95E1F7D60117963C934F
:102C90002E9316973BC090E005970E94D2080FC074
:102CA000E82FF0E0EE0FFF1FE55DF14F808191818D
:102CB0008051984F20C08091AD109091AE10F601D8
:102CC0009783868323C08091AF109091B01013C07A
:102CD0008091B1109091B210F2CF8091B310909189
:102CE000B41009C08091B5109091B610E8CF8091D2
:102CF000B7109091B810D60117969C938E931697A3
:102D000005C0F6018683178210922A0D80912A0D44
:102D10008F5F80932A0D8CE0DF91CF910F91EF9020
:102D2000DF90CF90089588EB93E00E946A080895A1
:102D3000CF93DF9380EF93E00E946A08C0E0D0E079
:102D400084EF93E00E946A08FE01E35AFF4E8081FF
:102D500090E00E94A0082196C031D10589F786EF46
:102D600093E00E946A08C0E0D0E084EF93E00E9404
:102D70006A08FE01EF58FF4E808190E00E94A00893
:102D80002196C031D10589F78DEF93E00E946A0842
:102D9000C0E0D0E084EF93E00E946A08FE01E75BA8
:102DA000FF4E808190E00E94A0082196C031D1059D
:102DB00089F784E094E00E946A0884EF93E00E941F
:102DC0006A0880E090E00E94D2080E94A00884EF88
:102DD00093E00E946A0881E090E00E94D2080E947D
:102DE000A00884EF93E00E946A0882E090E00E94CD
:102DF000D2080E94A00884EF93E00E946A0883E052
:102E000090E00E94D2080E94A0088BE094E00E940B
:102E10006A08C0E0D0E084EF93E00E946A08FE01F7
:102E2000EE0FFF1FEB57FF4E808191810E94A0089B
:102E30002196C031D10579F782E194E00E946A08B9
:102E4000C0E0D0E084EF93E00E946A08FE01EE0F3C
:102E5000FF1FE35CF14F808191810E94A0082196C1
:102E6000C830D10579F789E194E00E946A08809121
:102E7000E40D90E00E94A00884EF93E00E946A08AD
:102E80008091E00D9091E10D0E94A00884EF93E005
:102E90000E946A088091DE0D9091DF0D0E94A008CB
:102EA00084EF93E00E946A088091DD0D90E00E941B
:102EB000A00884EF93E00E946A088091E60D90914B
:102EC000E70DA091E80DB091E90D0E94A00884EFF4
:102ED00093E00E946A088091350E9091360EA09181
:102EE000370EB091380E0E94A00884EF93E00E9444
:102EF0006A088091E50D90E00E94A00881E294E0CC
:102F00000E946A08C0E0D0E084EF93E00E946A0863
:102F1000FE01EE0FFF1FE355FF4E808191810E945D
:102F2000A0082196CB30D10579F788E294E00E9481
:102F30006A08DF91CF9108950F931F93CF93DF938A
:102F40008FEF0E9460068FEF0E94600640E050E025
:102F500020E030E0F901EF58FF4E8081480F511D0D
:102F60002F5F3F4F20313105A9F7A4E056954795D3
:102F7000AA95E1F7842F0E94600640E050E020E02F
:102F800030E0F901E75BFF4E8081480F511D2F5F54
:102F90003F4F20313105A9F7F5E056954795FA9551
:102FA000E1F7842F0E946006C0E0D0E08E01000FA0
:102FB000111F0B571F4EF801808191818050984F4F
:102FC000892F0E946006F801808191810E9460062D
:102FD0002196C031D10551F7DF91CF911F910F910B
:102FE0000895CF93DF938FEF0E9460068FEF0E94CA
:102FF000600640E050E020E030E0F901EF58FF4E7D
:103000008081480F511D2F5F3F4F20313105A9F7B7
:1030100094E0569547959A95E1F7842F0E946006B3
:1030200040E050E020E030E0F901E75BFF4E8081B6
:10303000480F511D2F5F3F4F20313105A9F785E023
:10304000569547958A95E1F7842F0E946006C0E067
:10305000D0E0FE01EE0FFF1FEB57FF4E8081918104
:103060008050984F60E170E00E949624862F0E9465
:1030700060062196C031D10561F7DF91CF910895A7
:103080000F931F93DF93CF9300D00F92CDB7DEB78E
:103090008BE189838BE58A838AE48B838E010F5FC2
:1030A0001F4FC80163E00E94090682E089831A82EB
:1030B000C80162E00E9409060F900F900F90CF9117
:1030C000DF911F910F9108950F931F93DF93CF937B
:1030D00000D000D0CDB7DEB78BE189838BE58A8342
:1030E0008BE38B8388E48C838E010F5F1F4FC801B5
:1030F00064E00E94090682E089831A82C80162E0C6
:103100000E9409060F900F900F900F90CF91DF91C2
:103110001F910F9108951F93CF93DF930E94401842
:103120000E9464188CE294E00E946A0887E694E0AA
:103130000E946A0884E994E00E946A0880ED94E0A5
:103140000E946A088FED94E00E946A088091770ED1
:10315000803150F588EE94E00E946A088091780EE4
:1031600090E00E94A00880EF94E00E946A0880919D
:10317000770E90E001960E94A00881E095E00E9401
:103180006A088091790E90E00E94A00884E095E0A2
:103190000E946A0880917A0E90917B0E0E94A0088E
:1031A00086E095E00E946A088BE095E00E946A083C
:1031B00087E195E00E946A0881E295E00E946A0832
:1031C00083E395E00E946A0882E495E00E946A0821
:1031D00088E495E00E946A088EE495E00E946A08FF
:1031E00084E595E00E946A0881E295E00E946A0801
:1031F00088E695E00E946A08C0E0D0E013E0FE0196
:10320000EF58FF4E8081819FC00111248B55904063
:103210000E94A00887E795E00E946A082196C031C5
:10322000D10569F789E795E00E946A08C0E0D0E01F
:1032300013E0FE01E35AFF4E8081819FC0011124FB
:103240008B5590400E94A00887E795E00E946A088D
:103250002196C031D10569F789E995E00E946A0895
:10326000C0E0D0E013E0FE01E35AFF4E4081FE01D2
:10327000EF58FF4E8081819FC001112450E09A01D8
:10328000220F331F240F351F821B930B0E94A008AF
:1032900087E795E00E946A082196C031D10519F7A9
:1032A00089EB95E00E946A08C0E0D0E0FE01E75B90
:1032B000FF4E808190E00E94A00887E795E00E9481
:1032C0006A082196C031D10589F789ED95E00E9401
:1032D0006A088091E40D90E00E94A00889EF95E0D3
:1032E0000E946A088091E00D9091E10D0E94A00873
:1032F0008BEF95E00E946A088091DE0D9091DF0DC2
:103300000E94A0088DEF95E00E946A088091DD0D73
:1033100090E00E94A0088FEF95E00E946A088091DB
:10332000360D9091370D0E94A0088BEF95E00E941A
:103330006A0880912202909123020E94A00881E2F3
:1033400096E00E946A088091E60D9091E70DA091A9
:10335000E80DB091E90D0E94A00883E496E00E9478
:103360006A088091350E9091360EA091370EB0917B
:10337000380E0E94A00886E496E00E946A088091B8
:10338000E50D90E00E94A00887E696E00E946A089A
:1033900086E796E00E946A0880E090E00E94D208EA
:1033A0000E94A00887E896E00E946A0881E090E009
:1033B0000E94D2080E94A0088BE896E00E946A084A
:1033C00082E090E00E94D2080E94A0088FE896E078
:1033D0000E946A0883E090E00E94D2080E94A00840
:1033E00083E996E00E946A088AE996E00E946A08EA
:1033F0008091660090E00E94A00889EA96E00E9411
:103400006A0883EB96E00E946A088091390E90E08A
:103410000E94A00882EC96E00E946A0880913A0E11
:1034200090E00E94A00889EA96E00E946A0885EC74
:1034300096E00E946A0810E00FC0E12FF0E0EE0F66
:10344000FF1FEB57FF4E808191810E94A00887E704
:1034500095E00E946A081F5F8091DC0D181768F3E1
:1034600089EA96E00E946A0884ED96E00E946A0864
:103470008091D00D992787FD90950E94A00889EA38
:1034800096E00E946A0883EE96E00E946A0889EF3F
:1034900095E00E946A0880917C0E90E00E94A0084E
:1034A00082EF96E00E946A0880917C0E2091780E4F
:1034B00090E0820F911D0E94A00885EF96E00E9487
:1034C0006A0810E011C080917C0EE80FF11DEE0F2C
:1034D000FF1FEF56F14F808191810E94A00887E77E
:1034E00095E00E946A081F5F8091780E181750F4CB
:1034F000E12FF0E080917C0E9F01280F311D2034D8
:1035000031050CF388EF96E00E946A0889EF95E098
:103510000E946A088091820E90E00E94A00882EFCB
:1035200096E00E946A088091820E20917E0E90E0C3
:10353000820F911D0E94A00885EF96E00E946A0804
:1035400010E011C08091820EE80FF11DEE0FFF1FF9
:10355000EF56F14F808191810E94A00887E795E0A6
:103560000E946A081F5F80917E0E181750F4E12FA9
:10357000F0E08091820E9F01280F311D203431052B
:103580000CF389EA96E00E946A08DF91CF911F91BF
:1035900008950F93FC0101900020E9F73197E81B93
:1035A000F90BDB016D917C918E0F9F1F40E020E0B5
:1035B00001E00E94F7060F9108950F93FC0101901E
:1035C0000020E9F73197E81BF90BDB016D917C9145
:1035D0008E0F9F1F40E020E001E00E94F7060F9150
:1035E00008950F93FC0101900020E9F73197E81B43
:1035F000F90BDB016D917C918E0F9F1F40E020E065
:1036000001E00E94F7060F9108950F93DC010D90E1
:103610000020E9F71197A81BB90BFB016081772700
:1036200067FD70958A0F9B1F40E020E001E00E943B
:10363000F7060F9108950F93FC0101900020E9F720
:103640003197E81BF90BDB016C918E0F9F1F70E027
:1036500040E020E001E00E94F7060F9108958F926C
:103660009F92AF92BF92CF92DF92EF92FF920F9311
:103670001F93DF93CF93CDB7DEB7A0970FB6F89423
:10368000DEBF0FBECDBF282F19824091CB0D909188
:10369000CA0DA92FB0E0FD01ED50F34FE081BE2E21
:1036A000B40E8091830E882319F481E08093830EF9
:1036B000233309F46AC0243338F4213309F4ACC04D
:1036C000223309F0BCC013C0263329F1283321F07E
:1036D000243309F0B4C060C0442311F0415012C03B
:1036E000A250B34F8C9181508093CB0D10C0242FEA
:1036F00030E0A250B34F8C9190E001972817390722
:1037000024F44F5F4093CB0D02C01092CB0DB090CC
:10371000CB0DBE0E94C0AB2DB0E0FD01E553F84FCC
:10372000E081E230F9F0E33030F4EE23D9F0E1301B
:1037300009F085C008C0E430F9F0E430E8F0E53085
:1037400009F07DC022C0AA0FBB1FA45FB74FED9147
:10375000FC9180819181A281B3818C509E4FAF4FAB
:10376000BF4F4BC0AA0FBB1FA45FB74FED91FC9199
:10377000808191810A9630C0AA0FBB1FA45FB74F0A
:10378000ED91FC9180818F5F45C09A3010F49F5F6E
:1037900046C01092CA0D49C0AB2DB0E0FD01E55303
:1037A000F84FE081E23079F0E33030F4EE2359F065
:1037B000E13009F044C013C0E43021F1E43010F1ED
:1037C000E530E9F529C0AA0FBB1FA45FB74FED9103
:1037D000FC91808191810A979183808330C0AA0FE8
:1037E000BB1FA45FB74FED91FC9180819181A281B5
:1037F000B381845F9140A040B04080839183A283D5
:10380000B3831DC0AA0FBB1FA45FB74FED91FC91FE
:1038100080818150808313C0992321F0915090932F
:10382000CA0D03C08AE08093CA0D1092CB0DE091BF
:10383000CA0DF0E0ED50F34FB080B092CC0D0B2DDF
:1038400010E02091CC0D8091830E90E0820F911DAD
:103850000197081719074CF08091830E2B2D281B18
:10386000822F8F5F8093CC0D04C0B21610F4B092FB
:10387000CC0D80E197E00E946A08E091CA0DF0E06B
:10388000ED50F34F208181E090E0821B9109800F81
:10389000911F0E94A0088BEF95E00E946A08E091BA
:1038A000CA0DF0E0E250F34F808190E00E94A00842
:1038B00084E197E00E946A08E091CA0DF0E0EE0F03
:1038C000FF1FE352F34F808191810E946A0886E1D5
:1038D00097E00E946A088BE197E00E946A08E091F5
:1038E000CA0DF0E0EE0FFF1FE352F34F60817181CC
:1038F00085E190E10E944A2500E010E0C8018F5E5A
:10390000904F6DEF75E00E944A25065E1F4F31E033
:103910000430130799F7A090CC0D7E010894E11CA8
:10392000F11CEAE18E2E912C89C01982BA1429F477
:10393000C70163E377E00E943F258601000F111F56
:10394000F801E850F44F60817181C7010E943F2562
:10395000C70165E377E00E943F25F601E553F84F84
:10396000E081E23001F1E33028F4EE2351F0E13060
:10397000C1F510C0E43039F1E430F0F0E53089F5FC
:103980002BC0045F174FF80160817181C7010E944D
:10399000DD1A27C0045F174FF80160817181C701EC
:1039A0000E94C91A1EC0045F174FF801608171811F
:1039B000C7010E94F11A15C0045F174FF80160811A
:1039C0007181C7010CC0045F174FF80160817181DC
:1039D000C7010E94051B05C0C7016AEC7DE00E947B
:1039E0001B1B87E397E00E946A088091CC0D96012B
:1039F000281B3109C9010E94A00884E197E00E94B8
:103A00006A08C7010E946A088BE397E00E946A086F
:103A10008091CC0DF601E81BF109EA30F1056CF458
:103A2000188EE89DC001E99D900DF89D900D112420
:103A30008F5E904FB7010E944A25A394CA2CDD24C3
:103A40002091830E8091CC0D90E0820F911DC816BD
:103A5000D906A4F430E43A1588F0E091CA0DF0E0FC
:103A6000DF01A250B34F2C91ED50F34F808190E0D5
:103A7000820F911DC816D9060CF457CF8BE197E041
:103A80000E946A08A0960FB6F894DEBF0FBECDBFA5
:103A9000CF91DF911F910F91FF90EF90DF90CF902A
:103AA000BF90AF909F908F900895AF92BF92CF92AA
:103AB000DF92EF92FF920F931F93CF93DF931092B9
:103AC000CD0D1092CF0D80E090E02AE130E0829F92
:103AD000F001839FF00D929FF00D1124EF5EF04FE7
:103AE000108201968A30910591F79A9AA29A80E005
:103AF00090E0FC01EE0FFF1FEB57FF4E118210828A
:103B0000019680319105A9F780E090E020E80FB69A
:103B1000F89420936100809361000FBE399A419A16
:103B2000579A5F9A6B9A739804B603FC03C081E0BE
:103B30008093EC0D1092EC0D6E98769A60E076E929
:103B400080E090E00E94C1058EE397E00E946A0841
:103B500088EB93E00E946A0860E875E280E090E0FC
:103B60000E94E5050E94DF0A0E94C7080E949A038E
:103B70000E94B40980E00E942F1BAA24AA9401E0AD
:103B8000B3E0FB2EA4E0EA2EF4ECCF2EF9E0DF2E1A
:103B9000E2E0BE2E9091290DA092290D9F3F09F4DD
:103BA0005AC08091DB0D882309F055C0992309F490
:103BB00052C0892F0E942F1B80913C0E882309F14F
:103BC00010923C0E8BE697E00E946A0820E030E0FD
:103BD000F901EE0FFF1FEB57FF4E80819181F90134
:103BE000EE0FFF1FE35CF14F918380832F5F3F4F08
:103BF0002830310569F70E94050385E897E00E94A7
:103C00006A088091860E8823C1F01092860E83E99F
:103C100097E00E946A08F092770E10927C0EE09274
:103C20007D0E1092820ED092700EC0926F0E0E9486
:103C3000050385E897E00E946A088091850E882335
:103C400041F01092850E0E94050385E897E00E94DE
:103C50006A080093DB0DA8958091E30D882371F429
:103C60008091EA0D813051F08091EE0D813009F0A4
:103C7000D7C08091EB0D853009F0D2C01091E30DD3
:103C80001092E30D133619F4B092EB0D04C0123408
:103C900029F4F092EB0D0093EA0D52C01D3619F491
:103CA0001092EB0DF8CF1636C1F420E030E0F901A8
:103CB000EE0FFF1FEB57FF4E80819181F901EE0F50
:103CC000FF1FE35CF14F918380832F5F3F4F2830CC
:103CD000310569F70E94050333C0133721F0812FA6
:103CE00080538A3028F40093EB0D1092EA0D28C01F
:103CF000133529F40E94050388EA97E01FC01236A5
:103D000019F40E94AA001CC0153739F48091EA0DFD
:103D1000902F981B9093EA0D13C0123759F40E940C
:103D2000641884EB97E00E946A08F89480E00E948F
:103D3000EB03FFCF193421F488EB93E00E946A086B
:103D40008091EB0D823009F463C0833030F4882316
:103D500059F0813009F064C00AC0833009F45BC0B7
:103D6000843009F05DC05AC00E948B1859C0812F61
:103D70000E942F1B80913C0E882309F110923C0E6B
:103D80008BE697E00E946A0820E030E0F901EE0F30
:103D9000FF1FEB57FF4E80819181F901EE0FFF1F4E
:103DA000E35CF14F918380832F5F3F4F28303105D3
:103DB00069F70E94050385E897E00E946A088091F0
:103DC000860E8823C1F01092860E83E997E00E9448
:103DD0006A08F092770E10927C0EE0927D0E10929F
:103DE000820ED092700EC0926F0E0E94050385E87D
:103DF00097E00E946A088091850E882389F01092CE
:103E0000850E0E94050385E897E00E946A0808C0B5
:103E10000E94981605C00E94F11702C00E949C17CC
:103E2000669906C080EC97E00E946A080E94AA008A
:103E30008091DA0D882311F41092D90D90913B0EE8
:103E4000913009F0A7CE8091DA0D853608F4A2CE24
:103E50009093D90DC0E0D0E0FE01EE0FFF1FE35CB0
:103E6000F14F80819181FE01EE0FFF1FEB57FF4E56
:103E700091838083C53040F5DE01AB5CB14F58962D
:103E8000EC915897F0E0EE0FFF1FEB57FF4E60816B
:103E9000718190962C91882777FD8095982F3327F4
:103EA00027FD3095432F532F0E94632424E630E0F2
:103EB00040E050E00E94A924220F331F441F551FE9
:103EC0008C2FB9010E945A092196C830D10521F6DC
:103ED00061CEEF92FF920F931F937B018C0120E044
:103EE00030E040E05FE40E94392288238CF0C80172
:103EF000B70120E030E040E05FE40E94E1200E9452
:103F000069229B01AC01205030404040504806C01F
:103F1000C801B7010E9469229B01AC01B901CA0125
:103F20001F910F91FF90EF900895A0E0B0E0EBE9B2
:103F3000FFE10C94E624DC012B01FA019C91923004
:103F400008F439C1EB018881823008F433C1943020
:103F500069F4843009F02FC111969C9111978981E1
:103F6000981709F428C1ABE2BDE025C1843009F4FB
:103F700021C18230A9F4923009F01DC19A01AD012E
:103F800088E0EA010990AE01E90109929E018150A1
:103F9000C1F7E201898111969C918923818308C12F
:103FA000923009F407C112962D903C901397EB01C3
:103FB0008A819B811496AD90BD90CD90DC9017972F
:103FC000EC80FD800E811F819101281B390BB90106
:103FD00037FF04C066277727621B730B60327105B9
:103FE0000CF061C0121613066CF537014801062E5D
:103FF00004C096948794779467940A94D2F721E04A
:1040000030E040E050E004C0220F331F441F551F32
:104010006A95D2F721503040404050402E213F2138
:1040200040235123211531054105510521F021E09F
:1040300030E040E050E079018A01E628F7280829BD
:1040400019293CC0232BD1F1260E371E350146011C
:10405000062E04C096948794779467940A94D2F7B6
:1040600021E030E040E050E004C0220F331F441F45
:10407000551F6A95D2F721503040404050402A21C8
:104080003B214C215D21211531054105510521F0D0
:1040900021E030E040E050E059016A01A628B7284D
:1040A000C828D9280BC0821593052CF01C01AA241E
:1040B000BB24650103C0EE24FF24870111969C9167
:1040C000D20111968C91981709F445C0992339F0C3
:1040D000A80197012A193B094C095D0906C0A601F0
:1040E00095012E193F09400B510B57FD08C0118255
:1040F0003382228224833583468357831DC081E027
:1041000081833382228288279927DC01821B930BCB
:10411000A40BB50B84839583A683B7830DC0220FB0
:10412000331F441F551F2483358346835783828161
:1041300093810197938382832481358146815781BE
:10414000DA01C9010197A109B1098F5F9F4FAF4FF4
:10415000BF4328F30BC0918333822282EA0CFB1CFD
:104160000C1D1D1DE482F5820683178383E0808386
:10417000248135814681578157FF1AC0C901AA277A
:1041800097FDA095BA2F81709070A070B070569571
:10419000479537952795822B932BA42BB52B84839A
:1041A0009583A683B78382819381019693838283CB
:1041B000DF0101C0D201CD01CDB7DEB7E2E10C9441
:1041C0000225A0E2B0E0E7EEF0E20C94F22469836D
:1041D0007A838B839C832D833E834F835887E9E0CA
:1041E000EE2EF12CEC0EFD1ECE010196B7010E94C1
:1041F00092238E010F5E1F4FCE010596B8010E94DB
:1042000092238A8991E089278A8BC701B801AE0180
:10421000475E5F4F0E94951F0E94BD22A096E6E078
:104220000C940E25A0E2B0E0E8E1F1E20C94F22457
:1042300069837A838B839C832D833E834F83588746
:10424000F9E0EF2EF12CEC0EFD1ECE010196B70128
:104250000E9492238E010F5E1F4FCE010596B8017A
:104260000E949223C701B801AE01475E5F4F0E94D2
:10427000951F0E94BD22A096E6E00C940E25A0E2B8
:10428000B0E0E5E4F1E20C94E62469837A838B8361
:104290009C832D833E834F835887CE010196BE01B8
:1042A000675F7F4F0E949223CE010596BE016F5E2D
:1042B0007F4F0E9492239985923088F089898230BD
:1042C000C8F0943019F4823051F404C0843029F4D9
:1042D000923081F48BE29DE0C6C0923049F420E038
:1042E0009A858A89981321E02A87CE010996BBC056
:1042F000823049F420E09A858A89981321E02A8B3C
:10430000CE014196B0C02D843E844F8458886D887C
:104310007E888F88988CEE24FF248701AA24BB24F2
:10432000650140E050E060E070E0E0E0F0E0C101F5
:1043300081709070892BE9F0E60CF71C081D191D9F
:104340009A01AB012A0D3B1D4C1D5D1D80E090E0E4
:10435000A0E0B0E0E614F7040805190520F481E0B8
:1043600090E0A0E0B0E0BA01A901480F591F6A1F10
:104370007B1FAA0CBB1CCC1CDD1C97FE08C081E077
:1043800090E0A0E0B0E0A82AB92ACA2ADB2A319638
:10439000E032F10549F0660C771C881C991C569494
:1043A000479437942794C3CFFA85EA892B893C89AF
:1043B0008B859C85280F391F2E5F3F4F17C0CA0180
:1043C00081709070892B61F016950795F794E794AA
:1043D00080E090E0A0E0B0E8E82AF92A0A2B1B2B45
:1043E00076956795579547952F5F3F4F77FDE7CFB8
:1043F0000CC0440F551F661F771F17FD4160EE0C60
:10440000FF1C001F111F21503040403090E0590721
:1044100090E0690790E4790760F32B8F3C8FDB0114
:10442000CA018F779070A070B07080349105A1059B
:10443000B10561F447FD0AC0E114F104010511055D
:1044400029F0405C5F4F6F4F7F4F40781A8EFE1708
:1044500011F081E08A8F4D8F5E8F6F8F78A383E09C
:10446000898FCE0149960E94BD22A096E2E10C946C
:104470000225A8E1B0E0EFE3F2E20C94F2246983B4
:104480007A838B839C832D833E834F83588789E077
:10449000E82EF12CEC0EFD1ECE010196B7010E9414
:1044A00092238E010F5E1F4FCE010596B8010E9428
:1044B00092238985823040F08989823028F0C701B3
:1044C000B8010E940A2401C08FEF6896E6E00C94C0
:1044D0000E25ACE0B0E0EFE6F2E20C94F62469833E
:1044E0007A838B839C83CE010196BE016B5F7F4FE5
:1044F0000E9492238D81823061F1823050F18430AC
:1045000021F48E81882351F12EC02F81388537FD0B
:1045100020C06E812F3131051CF06623F9F023C0D5
:104520008EE190E0821B930B29853A854B855C8553
:1045300004C056954795379527958A95D2F76623F7
:10454000B1F050954095309521953F4F4F4F5F4FBB
:104550000EC020E030E040E050E009C02FEF3FEF18
:104560004FEF5FE704C020E030E040E050E8B901E1
:10457000CA012C96E2E00C941225DF92EF92FF9292
:104580000F931F93FC01E480F58006811781D18091
:104590008081823048F480E090E0A0E1B0E0E82A39
:1045A000F92A0A2B1B2BA5C0843009F49FC0823046
:1045B00021F4EE24FF24870105C0E114F104010574
:1045C000110519F4E0E0F0E096C0628173819FEF7D
:1045D000623879070CF05BC022E83FEF261B370BEF
:1045E0002A3131052CF020E030E040E050E02AC0D4
:1045F000B801A701022E04C0769567955795479597
:104600000A94D2F781E090E0A0E0B0E004C0880F07
:10461000991FAA1FBB1F2A95D2F70197A109B109BB
:104620008E219F21A023B1230097A105B10521F080
:1046300081E090E0A0E0B0E09A01AB01282B392B9B
:104640004A2B5B2BDA01C9018F779070A070B07094
:1046500080349105A105B10539F427FF09C0205C1C
:104660003F4F4F4F5F4F04C0215C3F4F4F4F5F4F55
:10467000E0E0F0E02030A0E03A07A0E04A07A0E444
:104680005A0710F0E1E0F0E079018A0127C06038B4
:10469000710564F5FB01E158FF4FD801C7018F7721
:1046A0009070A070B07080349105A105B10539F407
:1046B000E7FE0DC080E490E0A0E0B0E004C08FE32E
:1046C00090E0A0E0B0E0E80EF91E0A1F1B1F17FFE4
:1046D00005C016950795F794E794319687E01695EF
:1046E0000795F794E7948A95D1F705C0EE24FF2447
:1046F0008701EFEFF0E06E2F679566276795902FA3
:104700009F77D794DD24D7948E2F8695492F462BFB
:10471000582F5D29B701CA011F910F91FF90EF90AB
:10472000DF900895FC01DB01408151812281622FDD
:104730006F7770E0221F2227221F9381892F880F15
:10474000822B282F30E0991F9927991F11969C934F
:10475000119721153105A9F541155105610571051F
:1047600011F482E037C082E89FEF13969C938E93FA
:1047700012979A01AB0167E0220F331F441F551FA8
:104780006A95D1F783E08C930DC0220F331F441F2D
:10479000551F12968D919C911397019713969C9398
:1047A0008E931297203080E0380780E0480780E43D
:1047B000580758F314962D933D934D935C93179798
:1047C00008952F3F310579F44115510561057105B3
:1047D00019F484E08C93089564FF03C081E08C9306
:1047E00012C01C9210C02F57304013963C932E934A
:1047F000129783E08C9387E0440F551F661F771F45
:104800008A95D1F7706414964D935D936D937C9364
:10481000179708951F93DC01FB019C91923008F4D7
:1048200047C08081823008F443C0943051F411961F
:104830001C91843099F58181682F70E0611B7109AA
:104840003FC0843021F0923031F48230B9F181815F
:10485000882389F12DC011961C9111978230F1F0B7
:1048600081811817D9F412962D913C91139782816A
:1048700093818217930794F028173907BCF0149698
:104880008D919D910D90BC91A02D24813581468103
:104890005781281739074A075B0718F4112341F09D
:1048A0000AC082179307A407B50740F4112319F033
:1048B00061E070E005C06FEF7FEF02C060E070E084
:1048C000CB011F910895629FD001739FF001829FD9
:1048D000E00DF11D649FE00DF11D929FF00D839F8F
:1048E000F00D749FF00D659FF00D9927729FB00D2C
:1048F000E11DF91F639FB00DE11DF91FBD01CF013F
:1049000011240895AA1BBB1B51E107C0AA1FBB1F9E
:10491000A617B70710F0A61BB70B881F991F5A954B
:10492000A9F780959095BC01CD01089597FB092EBC
:1049300007260AD077FD04D0E5DF06D000201AF460
:10494000709561957F4F0895F6F7909581959F4FEB
:104950000895A1E21A2EAA1BBB1BFD010DC0AA1FC0
:10496000BB1FEE1FFF1FA217B307E407F50720F0D8
:10497000A21BB30BE40BF50B661F771F881F991F53
:104980001A9469F760957095809590959B01AC019C
:10499000BD01CF01089597FB092E05260ED057FDC6
:1049A00004D0D7DF0AD0001C38F4509540953095DC
:1049B00021953F4F4F4F5F4F0895F6F790958095A3
:1049C000709561957F4F8F4F9F4F08952F923F9223
:1049D0004F925F926F927F928F929F92AF92BF920F
:1049E000CF92DF92EF92FF920F931F93CF93DF93BB
:1049F000CDB7DEB7CA1BDB0B0FB6F894DEBF0FBE18
:104A0000CDBF09942A88398848885F846E847D8464
:104A10008C849B84AA84B984C884DF80EE80FD8066
:104A20000C811B81AA81B981CE0FD11D0FB6F894DC
:104A3000DEBF0FBECDBFED010895662777270C942A
:104A40008125FC0188279927E89421912032E9F3F8
:104A5000293010F02E30C8F32B3241F02D3239F4CA
:104A6000689404C00E945125820F911D219120530A
:104A70002A30C0F31EF4909581959F4F0895FB0155
:104A8000DC010D900020E9F7119701900D920020B4
:104A9000E1F70895FB01DC0101900D920020E1F7A0
:104AA00008957AE0979F902D879F802D910D112476
:104AB0000895DC01CB01FC01F999FECF06C0F2BDDF
:104AC000E1BDF89A319600B40D9241505040B8F7CC
:104AD0000895DC01CB0103C02D910E947425415043
:104AE0005040D0F70895262FF999FECF1FBA92BDF6
:104AF00081BD20BD0FB6F894FA9AF99A0FBE0196BF
:104B000008958F929F92AF92BF92CF92DF92EF92D1
:104B1000FF920F931F93CF93DF93EC015B0161151D
:104B2000710519F0FB0191838083F9908F2D90E03E
:104B30000E94EF26892BC9F7FDE2FF1621F4F990B8
:104B4000EE24E39405C02BE2F21609F4F990EE246A
:104B50008E0101501040C8016CEC70E043E050E061
:104B60000E94F726892B01F58E010E5F1F4FC801A9
:104B70006FEC70E045E050E00E94F726892B19F4B5
:104B80008E01095F1F4FA114B10419F0F5011183C3
:104B90000083E0FC04C070E090E080E814C070E0A6
:104BA00090E080E86FEF08C1C80164ED70E043E079
:104BB00050E00E94F726892B69F4A114B10429F46E
:104BC00070E090E080EC6FE7F7C02296F501D183AA
:104BD000C083F6CF8824992440E050E060E070E084
:104BE000EF2DE053EA30A0F5F2E0EF2A8E2D90E0B1
:104BF0009C0128703070E2FE06C0232B79F50894E2
:104C0000811C911C2BC0232B19F00894810891085A
:104C1000DB01CA0112E0880F991FAA1FBB1F1A955A
:104C2000D1F7480F591F6A1F7B1F440F551F661F7E
:104C3000771F4E0F511D611D711D483929E952071B
:104C400029E9620729E1720748F084E0E82A06C0F2
:104C5000EE3F31F4E3FC39C098E0E92AF990C0CF87
:104C6000E53311F0E53189F529912D3219F4E0E1B0
:104C7000EE2A05C02B3219F081E090E003C02991A3
:104C800082E090E0E22FE053EA3018F0C81BD90B25
:104C90001CC020E030E0FCE020383F075CF4C90194
:104CA000880F991F880F991F280F391F220F331F54
:104CB0002E0F311DE991E053EA3068F3E4FE03C0A2
:104CC000309521953F4F820E931ECE2CDD24E1FEC0
:104CD00007C0A114B10421F02197F501D183C0834D
:104CE000CB01BA010E9413277B018C01F3E0CF2294
:104CF000DD2423E0C216D10421F417FB109517F927
:104D0000109557016801C801B70120E030E040E08C
:104D100050E00E940F27882309F44AC097FE0DC077
:104D20002BEEE22E20E0F22E909481949108939441
:104D3000C0E2D0E000E010E012C093E0E92E91E084
:104D4000F92EF6CFF7012591359145915491C60181
:104D5000B5010E943F215B016C018C1A9D0A8C16E3
:104D60009D0684F7D595C7950F5F1F4F0630110537
:104D700029F08CEF9FEFE80EF91EF1CFC501D601A7
:104D80007C018D018C2D880F8D2D881F8F3F51F058
:104D9000C601B50120E030E040E050E00E940F275E
:104DA000882331F482E290E09093EA108093E91036
:104DB0007E2D9F2D802F612F272F392F482F562F83
:104DC000B901CA01DF91CF911F910F91FF90EF9030
:104DD000DF90CF90BF90AF909F908F9008959111EA
:104DE00083C0803219F089508550D0F70895FB01B7
:104DF000DC014150504088F08D9181341CF08B359E
:104E00000CF4805E659161341CF06B350CF4605ECF
:104E1000861B611171F3990B0895881BFCCF40D05C
:104E200008F481E00895E89409C097FB3EF490955A
:104E30008095709561957F4F8F4F9F4F9923A9F073
:104E4000F92F96E9BB279395F69587957795679502
:104E5000B795F111F8CFFAF4BB0F11F460FF1BC046
:104E60006F5F7F4F8F4F9F4F16C0882311F096E9D9
:104E700011C0772321F09EE8872F762F05C0662387
:104E800071F096E8862F70E060E02AF09A95660F40
:104E9000771F881FDAF7880F9695879597F90895F9
:104EA000990F0008550FAA0BE0E8FEEF161617063B
:104EB000E807F907C0F012161306E407F50798F0A3
:104EC000621B730B840B950B39F40A2661F0232BBC
:104ED000242B252B21F408950A2609F4A140A69538
:104EE0008FEF811D811D0895992788270895F894D3
:024EF000FFCFF2
:104EF200526561645F53657475703A20000A0D0053
:104F020057726F6E672045454D414749433A20002D
:104F12002F00B400000000000000000000000000AC
:104F2200000000000000000000000000000000007F
:104F32000000000064006400640064006400640017
:104F42006400640009120D0810040B0E021407011C
:104F52000F050C0009120D0810040B0E02140701B4
:104F62000F050C000A0A0A0A0A0A0A0A0A0A0A0AA7
:104F72000A0A0A0A14141414141414141414141417
:104F8200141414141E1E1E1E1E1E1E1E1E1E1E1E67
:104F92001E1E1E1E646464646464646464646464E7
:104FA20064646464000102030405060708090A0B2D
:104FB2000C0D0E0F0E0F14150C100B191A111612E0
:104FC2000D171318110C1A150F10130B0E180D16BE
:104FD2001719121414120D0F181316110C1A100BA4
:104FE2000E15191716130E140F181510190B0C1A8B
:104FF200120D171115101317120E0C1A0B0F110D9B
:10500200161814190E0F14150C100B191A1116126A
:105012000D17131819110C1A150B140F1810120E64
:10502200170D13161613180D170F100B190E121554
:1050320014110C1A0E17120F110C1A1510160B144C
:1050420019130D180B0C0D0E0F1011121314151647
:105052001718191A000102030405060745525231B6
:105062000D0A00455252320D0A00455252330D0AC2
:1050720000455252340D0A0054454D323A20002E5A
:10508200000A0D00505245323A200043414C493A41
:1050920020003B000305080E1A302E382D31333123
:1050A20030303632353734000A0D535953494E46A3
:1050B2004F3A7A69676269742F72782D70776D350D
:1050C2006334612F6D6573686E65746963732F3025
:1050D2002E382D313331303036323537340A0D0027
:1050E20053434E003B00200A0D52534900200A0D43
:1050F2004C514900200A0D41444300200A0D434807
:105102005600200A0D46535600200A0D4554433BD3
:1051120000200A0D47505300200A0D002D2D2D2D81
:105122002D2D2D2D2D2D2D2D2D2D2D2D2D2D2D2DAD
:105132002D2D2D2052434F50454E3234202D2D2DF2
:105142002D2D2D2D2D2D2D2D2D2D2D2D2D2D2D2D8D
:105152002D2D2D2D0A0D00496E666F3A202020203C
:1051620020202020205A6967626974205258203515
:105172004368616E6E656C2D536572766F2D505764
:105182004D0A0D0053797374656D3A20202020205A
:1051920020207A69676269742F72782D70776D3575
:1051A2006334612F6D6573686E65746963732F3044
:1051B2002E382D313331303036323537340A0D0046
:1051C2004472697665723A202020202020200070E7
:1051D200776D2D6F757420006E6175746963280098
:1051E2004368616E6E656C732D3E536572766F2DEA
:1051F200003B20007800757329200074656C656D92
:10520200657472696520006661696C7361766520F8
:1052120000202020202020202020202020202020AC
:105222000A0D0050726F746F636F6C202020202073
:1052320020006473737320006668737320007468BF
:10524200737320006C697374656E2D6265666F728C
:10525200652D74616C6B2000525353492864426D72
:10526200293A20202020002C00202020202020204D
:1052720020202020202020200A0D4E4F495345286F
:1052820064426D293A202020002020202020202066
:1052920020202020202020200A0D534E2D44696614
:1052A20066286442293A2020002020202020202045
:1052B20020202020202020200A0D4C51493A202075
:1052C20020202020202020200020202020202020FC
:1052D20020202020202020200A0D4552524F5253D8
:1052E2003A202020202020200028002F0020002506
:1052F20029202020202020202020202020202020A3
:105302000A0D484F50503A202020202020202020F3
:1053120000202020202020202020202020202020AB
:1053220020200A0D547849443A20202020202020B1
:10533200202000202800292020202020202020209A
:105342002020202020200A0D5345513A20202020E1
:10535200202020202020002020202020202020206B
:105362002020200A0D0041444327733A20202020A8
:1053720020202020303D0020313D0020323D002001
:10538200333D00202020200A0D004F534343414C5F
:10539200202020202020202000202020202020202B
:1053A2000A0D005461626C65733A2020202020208F
:1053B20020002C200056616C75657320202020206F
:1053C200202020004C6173742D4D756C74694E75EC
:1053D2006D20004D756C746976616C756573202063
:1053E20020002D3E00292000202020202020200AFD
:1053F2000D4D756C746976616C7565733220200091
:105402004D543A003A0020200A0D002D2D2D2D2D4D
:105412002D2D2D2D2D2D2D2D2D2D2D2D2D2D2D2DBA
:105422000A0D003E003D004D453A000A0D00726330
:105432006F70656E32342D727820285A69676269FE
:105442007420525820354368616E6E656C2D536529
:1054520072766F2D50574D290A0D00536574746989
:105462006E672046616C65736176652D56616C7559
:1054720065730A0D0053657475702D53617665640A
:105482000A0D004D756C746970726F702D536574DE
:1054920074696E67730A0D002E2E2E736176656431
:1054A2002E2E2E002E2E2E72657365742E2E2E0039
:1054B20062696E642E2E2E2E0A0D00010303030371
:1054C20000000000000000000303030303030303C2
:1054D200040404040404040404040404040404048A
:1054E2000404040404040404020203020203030386
:1054F200030203030303020303030303350E390EFE
:105502003A0E3B0E3C0E3D0E3F0E410E430E450E33
:10551200470E490E4B0E4D0E4E0E4F0E500E510EB3
:10552200520E530E540E550E560E570E580E590E5D
:105532005A0E5B0E5C0E5D0E5E0E5F0E600E610E0D
:10554200620E630E640E650E660E670E680E690EBD
:105552006A0E6B0E6C0E6D0E6F0E710E720E740E65
:10556200760E770E780E790E7A0E7C0E7D0E7E0EFA
:105572007F0E800E820E830E840E850E860E696467
:10558200007461626C650074696D657461626C655A
:10559200004661696C736176654D6F6465004661B2
:1055A200696C73617665536574004661696C7361F9
:1055B200766556616C7565735F31004661696C731F
:1055C20061766556616C7565735F32004661696C20
:1055D2007361766556616C7565735F330046616908
:1055E2006C7361766556616C7565735F34004661F4
:1055F200696C7361766556616C7565735F350046DB
:1056020061696C7361766556616C7565735F3600AE
:105612004661696C7361766556616C7565735F3757
:10562200004661696C7361766556616C7565735F7E
:105632003800536572766F4D61705F310053657249
:10564200766F4D61705F3200536572766F4D617097
:105652005F3300536572766F4D61705F340053653E
:1056620072766F4D61705F3500536572766F4D6172
:10567200705F3600536572766F4D61705F3700530D
:105682006572766F4D61705F3800536572766F4454
:1056920075616C526174655F3100536572766F4457
:1056A20075616C526174655F3200536572766F4446
:1056B20075616C526174655F3300536572766F4435
:1056C20075616C526174655F3400536572766F4424
:1056D20075616C526174655F3500536572766F4413
:1056E20075616C526174655F3600536572766F4402
:1056F20075616C526174655F3700536572766F44F1
:1057020075616C526174655F3800536572766F41E2
:10571200747655705F3100536572766F41747655B9
:10572200705F3200536572766F41747655705F33E5
:1057320000536572766F41747655705F340053651D
:1057420072766F41747655705F3500536572766F6D
:1057520041747655705F3600536572766F41747688
:1057620055705F3700536572766F41747655705F7E
:105772003800536572766F417476446F776E5F318D
:1057820000536572766F417476446F776E5F3200B4
:10579200536572766F417476446F776E5F33005350
:1057A2006572766F417476446F776E5F340053652D
:1057B20072766F417476446F776E5F35005365720F
:1057C200766F417476446F776E5F360053657276FA
:1057D2006F417476446F776E5F3700536572766FF0
:1057E200417476446F776E5F380050574D52617442
:1057F200655F310050574D526174655F3200505001
:105802004D4368616E6E656C730050504D53796EF6
:10581200630050504D53686966740050504D496E94
:1058220076657274006D756C74695F6368616E6E23
:10583200656C006D756C74695F6368616E6E656C32
:1058420073006D756C74695F6D73796E635F6E75ED
:105852006D006D756C74695F6D73796E635F6C65F5
:105862006E006D756C74695F6368616E6E656C6DF8
:105872006170006D756C7469325F6368616E6E652C
:105882006C006D756C7469325F6368616E6E656C15
:1058920073006D756C7469325F6D73796E635F6EE0
:1058A200756D006D756C7469325F6D73796E635FCF
:1058B2006C656E006D756C7469325F6368616E6EE3
:1058C200656C6D6170006D656E755F6C656E006311
:1058D20073765F6F75747075740073617665006DB1
:1058E200756C7469736574008E0891089708A10835
:1058F200AE08BA08CB08DC08ED08FE080F0920093B
:10590200310942094D09580963096E097909840967
:105912008F099A09AA09BA09CA09DA09EA09FA0928
:105922000A0A1A0A270A340A410A4E0A5B0A680A54
:10593200750A820A910AA00AAF0ABE0ACD0ADC0AD7
:10594200EB0AFA0A040B0E0B1A0B220B2B0B350B6C
:10595200430B520B620B720B830B920BA20BB30B1A
:10596200C40BD60BDF0BEA0BEF0B476C6F62616C5B
:10597200004661696C7361766500536572766F2DBE
:105982004D6170004475616C72617465004174769A
:105992002D5570004174762D446F776E0050574D2F
:1059A2002D4F75747075740050504D2D4F75747075
:1059B2007574004D756C746970726F70004D756C02
:1059C200746970726F7032004D656E75007A0C8169
:1059D2000C8A0C940C9D0CA40CAD0CB80CC30CCD11
:1059E2000CD80C00030D151D252D2F33383D030A4D
:1059F200080808080204050504010101010101016A
:105A02000101010101010101010101010101010184
:105A1200010101010101010101FF0100000000007B
:045A22000000000080
:00000001FF
